:0200000480007A
:100000009710000093800000171100001301810277
:1000100083A1000013020000930210001303F0FFFD
:10002000B70300809383F3FF3704008033824100DD
:10003000B382510033836100B38371003384810044
:100040002320310023224100232451002326610074
:1000500023287100232A8100971000009380C0FAA2
:1000600017110000130181FE03A400009304000097
:10007000130510009305F0FF370600801306F6FF06
:10008000B7060080B30494003305A400B305B400A0
:100090003306C400B306D40023208100232291003C
:1000A0002324A1002326B1002328C100232AD10044
:1000B00097100000938080F517110000130181FA5A
:1000C00083A6000013070000930710001308F0FF39
:1000D000B70800809388F8FF370900803387E6006F
:1000E000B387F60033880601B388160133892601E9
:1000F0002320D1002322E1002324F1002326010143
:1001000023281101232A210197100000938040F039
:1001100017110000130181F603A9000093090000E4
:10012000130A1000930AF0FF370B0080130BFBFF3C
:10013000B70B0080B3093901330A4901B30A5901E9
:10014000330B6901B30B79012320210123223101F3
:10015000232441012326510123286101232A71010F
:1001600097100000938000EB17110000130181F23B
:1001700083AB0000130C0000930C1000130DF0FF74
:10018000B70D0080938DFDFF370E0080338C8B01FF
:10019000B38C9B01338DAB01B38DBB01338ECB018F
:1001A0002320710123228101232491012326A1010F
:1001B0002328B101232AC101971C0000938CCCE5B0
:1001C000171D0000130D8DEE03AE0C00930D1000F3
:1001D000B30EBE01338FBE01B30FBF01B380BF01A9
:1001E0003381B001B301B1012320BD012322CD0130
:1001F0002324DD012326ED012328FD01232A1D00F0
:10020000232C2D00232E3D0097100000938000E149
:1002100017110000130181EB03AE0000B79DFFF73B
:10022000938D8D813300BE012320010097100000C3
:10023000938000DF17110000130181E903AE000075
:10024000B79DFFF7938D8D813300BE01B30200008F
:10025000232001002322510097100000938080DCAE
:1002600017110000130141E783A100003382010050
:10027000B30202003303500033070300B307070043
:1002800033880700B30C0001330D9001B30D0D004E
:10029000232041002322A1012324B10117150000CE
:1002A000130545D9971500009385C5E3370610F06F
:1002B0001306C6F26306B5028326C5002320D600C6
:1002C000832685002320D600832645002320D600E0
:1002D000832605002320D600130505016FF09FFD3E
:1002E000370510F0130505F223200500000000007B
:0402F000000000000A
:101000000000000001000000FFFFFFFFFFFFFF7F67
:1010100000000080CDAB00007856341298BADCFE98
:10102000145892360000000000000000000000008C
:10103000FFFFFFFFFFFFFFFFFFFFFFFFFFFFFFFFC0
:10104000FFFFFFFFFFFFFFFFFFFFFFFFFFFFFFFFB0
:10105000FFFFFFFFFFFFFFFFFFFFFFFFFFFFFFFFA0
:10106000FFFFFFFFFFFFFFFFFFFFFFFFFFFFFFFF90
:10107000FFFFFFFFFFFFFFFFFFFFFFFFFFFFFFFF80
:10108000FFFFFFFFFFFFFFFFFFFFFFFFFFFFFFFF70
:10109000FFFFFFFFFFFFFFFFFFFFFFFFFFFFFFFF60
:1010A000FFFFFFFFFFFFFFFFFFFFFFFFFFFFFFFF50
:1010B000FFFFFFFFFFFFFFFFFFFFFFFFFFFFFFFF40
:1010C000FFFFFFFFFFFFFFFFFFFFFFFFFFFFFFFF30
:1010D000FFFFFFFFFFFFFFFFFFFFFFFFFFFFFFFF20
:040000058000000077
:00000001FF
